:020000040000FA
:06000000B0EF18F0120041
:060008005EEF12F0120091
:06002A000300A2310000FA
:100030000F01000002000000A03100000D010000CF
:10004000020000008C3100000000000014000000DD
:100050008A6A896AF90E926E010EC26E0E0EC16E28
:10006000860EC06E010E066E0001640EEA6FD00EA1
:10007000ED6F070EEE6F080EEB6F0B0EEC6F000EC0
:10008000036E046A096E0A6A076E086A120099EC28
:1000900017F0060E0001FB5D31E36D50020B01E02D
:1000A00012000101105129E004010C51800B25E1DF
:1000B000400EE66E600EE66E000EE66E33EC16F055
:1000C000E552E552E5520101106B016A0250015CF4
:1000D00013E20150EA6AE00FE96E000EEA22EF50E7
:1000E000E66E0150EA6A600FE96E000EEA22E55200
:1000F000E750EF6E012AEAD7026A01D81200D9CF81
:10010000E6FFE1CFD9FF070EE12601010F51005CA8
:1001100002E30AEF12F00101105102E00AEF12F0BF
:100120000050EA6AA00FE96E000EEA22EF50F10AD1
:1001300002E1BEEF11F0010A02E181EF11F0020AC3
:1001400002E17FEF11F0C70A02E12DEF11F0010A81
:1001500002E1B6EF10F0070A02E135EF10F0010AF4
:1001600002E1FCEF0FF0030A02E1C6EF0FF0010A13
:1001700002E18FEF0FF01F0A02E141EF0FF0020AD8
:1001800002E1AEEF0EF0030A02E1EBEF0DF0020A1E
:1001900002E112EF0DF0070A02E1B5EF0CF0010ADF
:1001A00002E160EF0CF0030A02E10DEF0CF0010A2E
:1001B00002E18BEF0BF00F0A02E10AEF0BF0010AEC
:1001C00002E1AEEF0AF0030A02E166EF0AF0010A6B
:1001D00002E1FFEF09F0070A02E1C8EF09F0010AA6
:1001E00002E191EF09F0030A02E14AEF09F0010A86
:1001F00002E1C7EF07F03F0A02E195EF07F0010ABD
:1002000002E17BEF07F0030A02E15FEF07F0010A6A
:1002100002E145EF07F0070A02E129EF07F0010AC2
:1002200002E10BEF07F0030A02E1EFEF06F0010A2B
:1002300002E1D5EF06F00F0A02E18CEF06F0010AA9
:1002400002E173EF06F0030A02E128EF06F0010A6B
:1002500002E1DFEF05F0070A02E181EF05F0010A94
:1002600001E1F0D3030A01E192D3010A01E176D35F
:100270001F0A01E1F7D2010A01E1A8D2030A01E154
:100280001BD2010A01E1F7D1070A01E1C5D1010A38
:1002900001E1AAD1030A01E191D1010A01E178D17A
:1002A0000F0A01E1F7D0010A01E1E8D0030A01E1F8
:1002B000BFD0010A01E199D0070A65E0010A42E0D6
:1002C000030A0AE0010A02E004EF12F0E66A29ECF0
:1002D00012F0E55209EF12F0010EE66E29EC12F071
:1002E000E552B6DEE66A29EC12F0E552050EE66E3E
:1002F00029EC12F0E552E66A29EC12F0E552E66AC2
:1003000029EC12F0E552E66A29EC12F0E552010EF2
:10031000E66E29EC12F0E552200EE66E29EC12F0A2
:10032000E552520EE66E29EC12F0E552530EE66EDF
:1003300029EC12F0E552540EE66E29EC12F0E5526B
:1003400009EF12F0020EE66E29EC12F0E552E66AB1
:1003500029EC12F0E552050EE66E29EC12F0E5529A
:10036000E66A29EC12F0E552E66A29EC12F0E55251
:10037000E66A29EC12F0E552010EE66E29EC12F065
:10038000E55209EF12F0030EE66E29EC12F0E55289
:100390000028166E01010F51165C18E2002A005069
:1003A000EA6AA00FE96E000EEA22EFCFDFFF340EFB
:1003B000DF5C06E2DFCFE6FF29EC12F0E55205D064
:1003C000FE0EE66E29EC12F0E5520DD0FE0EE66E42
:1003D00029EC12F0E5520028EA6AA00FE96E000E3F
:1003E000EA22040EEF6E09EF12F0400E015C09E202
:1003F0000150EA6A600FE96E000EEA22EF6A012AF4
:10040000F4D7016A04010CBF0CD0400EE66E600EFA
:10041000E66E000EE66E33EC16F0E552E552E5525C
:1004200003D00101010E106F0FC100F009EF12F0AF
:10043000050EE66E29EC12F0E552000E036E046A1A
:10044000096E0A6A076E086A840ECB6E040ECA6EC5
:100450000B0EBC6EB80EBB6E9E9C9D8CBE6A0C0EC5
:10046000BD6E9494B36AB26A890EB16E0B0EBA6E09
:10047000C00EF26E1E0ED26E09EF12F0060EE66E80
:1004800029EC12F0E5529D9CBA6ABD6A0E0ED26E3E
:1004900009EF12F0070EE66E29EC12F0E552030E9A
:1004A0000024166E01010F51165C63E2002A005011
:1004B000EA6AA00FE96E000EEA22EF500D6E0D50B1
:1004C000030A40E0010A2BE0030A16E0010A01E0FA
:1004D0004CD0002A0050EA6AA00FE96E000EEA2212
:1004E000EF50066E002A0050EA6AA00FE96E000E77
:1004F000EA22EFCFEAF03CD0002A0050EA6AA00FCF
:10050000E96E000EEA22EFCFEEF0002A0050EA6A10
:10051000A00FE96E000EEA22EFCFEDF029D0002AFD
:100520000050EA6AA00FE96E000EEA22EFCFF0F069
:10053000002A0050EA6AA00FE96E000EEA22EFCF0F
:10054000EFF016D0002A0050EA6AA00FE96E000E04
:10055000EA22EFCFEBF0002A0050EA6AA00FE96E22
:10056000000EEA22EFCFECF003D0020E002600D0FE
:100570000DD0FE0EE66E29EC12F0E5520028EA6A74
:10058000A00FE96E000EEA22040EEF6E09EF12F0E2
:10059000080EE66E29EC12F0E552F29E06500D6E42
:1005A0000D5009E000000000000000000000000005
:1005B00000000D06F5D7F28E09EF12F0090EE66E77
:1005C00029EC12F0E552F29EEAC00DF00D5009E060
:1005D00000000000000000000000000000000D0608
:1005E000F5D7F28E09EF12F00A0EE66E29EC12F042
:1005F000E552F29EEDC012F0EEC013F0125013104F
:1006000008E000000000000000001206000E135A6F
:10061000F5D7F28E09EF12F00B0EE66E29EC12F010
:10062000E5520028166E01010F51165C15E2002AF2
:100630000050EA6AA00FE96E000EEA22EF500D6E3C
:100640000D5009E000000000000000000000000064
:1006500000000D06F5D70DD0FE0EE66E29EC12F067
:10066000E5520028EA6AA00FE96E000EEA22040EA5
:10067000EF6E09EF12F0A1940C0EE66E29EC12F069
:10068000E552C282C2B2FED7A1A40AD0E66A29EC22
:1006900012F0E552E66A29EC12F0E55209EF12F089
:1006A000C450E66E29EC12F0E552C350E66E29EC18
:1006B00012F0E55209EF12F00D0EE66E29EC12F081
:1006C000E5520028166E01010F51165C70E29D5034
:1006D000400B03E0D250200B06E1FE0EE66E29EC43
:1006E00012F0E55263D0A194002A0050EA6AA00FEC
:1006F000E96E000EEA22EF50126E136A12C00BF080
:1007000013C00CF0070E0C02F3CF0CF0070E0B0217
:10071000F3CF0BF0F4500C260F0E0D6EE80E126E98
:10072000030E136E1250131008E0000000000000CA
:1007300000001206000E135AF5D70D06083404E225
:1007400007500E08000E085408E3D880085004E74C
:10075000F20E075CFF0E085802E20D50DFE1A1A483
:1007600005D0E66A29EC12F0E55220D0083404E204
:1007700007500E08000E085408E3D880085004E71C
:10078000F20E075CFF0E085806E2FE0EE66E29EC3C
:1007900012F0E5520BD00050EA6AA00FE96E000E8D
:1007A000EA22EF50E66E29EC12F0E5520DD0FE0E73
:1007B000E66E29EC12F0E5520028EA6AA00FE96E15
:1007C000000EEA22040EEF6E09EF12F00E0EE66E36
:1007D00029EC12F0E5520028166E01010F51165C4B
:1007E00032E2002A0050EA6AA00FE96E000EEA2207
:1007F000EF500D6E010E0D1402E0000E01D0010E3F
:10080000E8B08B82E8A08B92020E0D1402E0010E7C
:1008100001D0000EE8B09482E8A09492040E0D146A
:1008200002E0010E01D0000EE8B08B80E8A08B90B2
:10083000080E0D1402E0010E01D0000EE8B0948005
:10084000E8A094900DD0FE0EE66E29EC12F0E55271
:100850000028EA6AA00FE96E000EEA22040EEF6E8D
:1008600009EF12F00F0EE66E29EC12F0E5520028A7
:10087000166E01010F51165C62E2002A0050EA6A0E
:10088000A00FE96E000EEA22EF50010B02E0010E0C
:1008900001D0000EE8B08A8AE8A08A9A0050EA6A7D
:1008A000A00FE96E000EEA22EF50020B02E0010EEB
:1008B00001D0000EE8B0938AE8A0939A0050EA6A4B
:1008C000A00FE96E000EEA22EF50040B02E0010EC9
:1008D00001D0000EE8B08A8CE8A08A9C0050EA6A39
:1008E000A00FE96E000EEA22EF50080B02E0010EA5
:1008F00001D0000EE8B0938CE8A0939C0050EA6A07
:10090000A00FE96E000EEA22EF50100B02E0010E7C
:1009100001D0000EE8B08A8EE8A08A9E0050EA6AF4
:10092000A00FE96E000EEA22EF50200B02E0010E4C
:1009300001D0000EE8B0938EE8A0939E0DD0FE0E7D
:10094000E66E29EC12F0E5520028EA6AA00FE96E83
:10095000000EEA22040EEF6E09EF12F0100EE66EA2
:1009600029EC12F0E5520D6A8ABA0D8093BA0D8215
:100970008ABC0D8493BC0D868ABE0D8893BE0D8AF9
:100980000D50E66E29EC12F0E55209EF12F0110E4F
:10099000E66E29EC12F0E552020E0024166E0101FB
:1009A0000F51165C40E2002A0050EA6AA00FE96E7F
:1009B000000EEA22EFCF13F0002A0050EA6AA00FDF
:1009C000E96E000EEA22EFCF12F0F29E8A9A8A8C2C
:1009D0008A9C8A8C8A9C8A8C8A9C8A8C8A9C8A8C27
:1009E0008A9C8A8C8A9C06500D6E0D5009E000008E
:1009F0000000000000000000000000000D06F5D718
:100A00008A8C8A9C0F0E0D6E0D4E08D01332123256
:100A1000819AD8B0818A818C819CF6D78A9A8A8CF7
:100A20008A9CF28E0DD0FE0EE66E29EC12F0E55295
:100A30000028EA6AA00FE96E000EEA22040EEF6EAB
:100A400009EF12F0120EE66E29EC12F0E552020EDA
:100A50000024166E01010F51165C44E2002A00507A
:100A6000EA6AA00FE96E000EEA22EFCF13F0002A27
:100A70000050EA6AA00FE96E000EEA22EFCF12F0F2
:100A8000F29E8A9A8A8C8A9C00008A8A8A8C8A9C26
:100A900000008A9A8A8C8A9C8A8C8A9C8A8C8A9C7E
:100AA0008A8C8A9C06500D6E0D5009E000000000F3
:100AB000000000000000000000000D06F5D78A8C41
:100AC0008A9C0F0E0D6E0D4E08D013321232819A91
:100AD000D8B0818A818C819CF6D78A9A8A8C8A9C2C
:100AE000F28E0DD0FE0EE66E29EC12F0E5520028D3
:100AF000EA6AA00FE96E000EEA22040EEF6E09EF1B
:100B000012F0130EE66E29EC12F0E5520028166E74
:100B100001010F51165C44E2002A0050EA6AA00F5E
:100B2000E96E000EEA22EFCF12F0F29E8A8A8A8CDA
:100B30008A9C8A8C8A9C00008A9A8A8C8A9C8A8CDD
:100B40008A9C8A8C8A9C8A8C8A9C06500D6E0D50D9
:100B500009E00000000000000000000000000000AC
:100B60000D06F5D78A8C8A9C090E0D6E0D4E07D0A6
:100B70001232819AD8B0818A818C819CF7D78A9A67
:100B80008A8C8A9C8A8C8A9C8A8C8A9C8A8C8A9C75
:100B90008A8C8A9C8A8C8A9C8A8C8A9CF28E0DD044
:100BA000FE0EE66E29EC12F0E5520028EA6AA00F6C
:100BB000E96E000EEA22040EEF6E09EF12F0140E39
:100BC000E66E29EC12F0E552F29E8A9A8A8C8A9C93
:100BD0008A8C8A9C00008A8A8A8C8A9C00008A9A65
:100BE0008A8C8A9C8A8C8A9C8A8C8A9C938A0650DE
:100BF0000D6E0D5009E00000000000000000000034
:100C0000000000000D06F5D78A8C8A9C0F0E0D6E31
:100C10000D4E08D08A8C8A9CD89081BAD880133225
:100C20001232F6D7D89013321232D89013321232D1
:100C30008A8C939A8A9CF28E13C0E6FF29EC12F0FC
:100C4000E55212C0E6FF29EC12F0E55209EF12F06E
:100C5000150EE66E29EC12F0E552F29E8A8A8A8C15
:100C60008A9C00008A9A8A8C8A9C00008A8A8A8CD4
:100C70008A9C00008A9A8A8C8A9C8A8C8A9C8A8C9C
:100C80008A9C938A06500D6E0D5009E0000000000A
:100C9000000000000000000000000D06F5D78A8C5F
:100CA0008A9C090E0D6E0D4E07D08A8C8A9CD890B6
:100CB00081BAD8801232F7D78A8C8A9C8A8C8A9C17
:100CC0008A8C8A9C8A8C8A9C8A8C8A9C8A8C8A9C34
:100CD0008A8C939A8A9CF28E12C0E6FF29EC12F05D
:100CE000E55209EF12F0160EE66E29EC12F0E5520D
:100CF000F29E8A9A8A8C8A9C00008A8A8A8C8A9CB4
:100D00008A8C8A9C8A9A8A8C8A9C8A8C8A9C8A8CF5
:100D10008A9CF28E09EF12F0170EE66E29EC12F0A3
:100D2000E5520028166E01010F51165C2FE2F29E6B
:100D3000002A0050EA6AA00FE96E000EEA22EFCF07
:100D400012F00001125020E08A9A8A8C8A9C0000DE
:100D50008A8A8A8C8A9C8A8C8A9C8A9A8A8C8A9CA7
:100D60008A8C8A9C8A8C8A9C06500D6E0D5009E0F4
:100D700000000000000000000000000000000D0660
:100D8000F5D700011206DDD7F28E0DD0FE0EE66E0D
:100D900029EC12F0E5520028EA6AA00FE96E000E75
:100DA000EA22040EEF6E09EF12F0180EE66E29EC3F
:100DB00012F0E552F29E8A9A8A8C8A9C8A8C8A9CCE
:100DC0008A8C8A9C00008A8A8A8C8A9C00008A9A73
:100DD0008A8C8A9C8A8C8A9CF28E09EF12F0190EFA
:100DE000E66E29EC12F0E552F29E8A8A8A8C8A9C81
:100DF00000008A9A8A8C8A9C8A8C8A9C00008A8A43
:100E00008A8C8A9C00008A9A8A8C8A9C8A8C8A9C0A
:100E1000F28E09EF12F01A0EE66E29EC12F0E5528E
:100E2000F29E8A9A8A8C8A9C00008A8A8A8C8A9C82
:100E300000008A9A8A8C8A9C00008A8A8A8C8A9C02
:100E400000008A9A8A8C8A9C8A8C8A9CF28E09EF8E
:100E500012F01B0EE66E29EC12F0E552F29E8A8A21
:100E60008A8C8A9C8A8C8A9C00008A9A8A8C8A9CAA
:100E700000008A8A8A8C8A9C00008A9A8A8C8A9CC2
:100E80008A8C8A9CF28E09EF12F01C0EE66E29EC19
:100E900012F0E552F29E8A9A8A8C8A9C00008A8A15
:100EA0008A8C8A9C8A8C8A9C8A8C8A9C00008A9A6A
:100EB0008A8C8A9C8A8C8A9CF28E09EF12F01D0E15
:100EC000E66E29EC12F0E552F29E8A8A8A8C8A9CA0
:100ED00000008A9A8A8C8A9C8A8C8A9C8A8C8A9C3A
:100EE00000008A8A8A8C8A9C00008A9A8A8C8A9C52
:100EF000F28E09EF12F01E0EE66E29EC12F0E552AA
:100F0000F29E8A9A8A8C8A9C8A8C8A9C8A8C8A9C79
:100F100000008A8A8A8C8A9C8A8C8A9C00008A9A21
:100F20008A8C8A9CF28E09EF12F01F0EE66E29EC75
:100F300012F0E5520028166E01010F51165C18E2FE
:100F4000002A0050EA6AA00FE96E000EEA22EFCFF5
:100F500012F0F29E070E0D6E0D4E07D01232819ADE
:100F6000D8B0818A818C819CF7D78A9AF28E0DD075
:100F7000FE0EE66E29EC12F0E5520028EA6AA00F98
:100F8000E96E000EEA22040EEF6E09EF12F0200E59
:100F9000E66E29EC12F0E552020E0024166E0101F5
:100FA0000F51165C01E367D1002A0050EA6AA00FD6
:100FB000E96E000EEA22EFCF13F0002A0050EA6A31
:100FC000A00FE96E000EEA22EFCF12F0010E12C060
:100FD000DBFF020E13C0DBFFF29E8A9A8A8C8A9C8A
:100FE00000008A8A8A8C8A9C00008A9A8A8C8A9C51
:100FF0008A8C8A9C8A8C8A9C8A8C8A9C06500D6E6C
:101000000D5009E00000000000000000000000009A
:1010100000000D06F5D78A8C8A9C0F0E0D6E0D4EC2
:1010200008D013321232819AD8B0818A818C819C87
:10103000F6D78A9A8A8C8A9C030EDB6A040EDB6AD6
:10104000030EDBCF16F0040EDBCF17F00001EB51DF
:10105000000117AE02D0D89003D0165C000E1758CE
:1010600001E398D08A9A8A8C8A9C8A8C8A9C8A8C82
:101070008A9C00008A8A8A8C8A9C00008A9A8A8CC0
:101080008A9C8A8C8A9CEAC00DF00D5009E0000011
:101090000000000000000000000000000D06F5D771
:1010A0008A9A8A8C8A9C00008A8A8A8C8A9C8A8C7A
:1010B0008A9C8A8C8A9C00008A9A8A8C8A9C8A8C58
:1010C0008A9C06500D6E0D5009E0000000000000E3
:1010D00000000000000000000D06F5D78A9A8A8CF7
:1010E0008A9C8A8C8A9C00008A8A8A8C8A9C00004E
:1010F0008A9A8A8C8A9C8A8C8A9C8A8C8A9C938AFB
:1011000006500D6E0D5009E00000000000000000C8
:101110000000000000000D06F5D78A8C8A9C0F0E97
:101120000D6E0D4E08D08A8C8A9CD89081BAD880DA
:1011300013321232F6D7D89013321232D8901332BB
:1011400012328A8C939A8A9C06500D6E0D5009E0DB
:1011500000000000000000000000000000000D067C
:10116000F5D7010EDBCF16F0020EDBCF17F01250D1
:10117000161802E11350171807E1030EDB500D6E2D
:10118000030EDB68040EDB6A030EDB2A040E01E3A8
:10119000DB2A56D7F28EF29ED950030FE96EDACFD2
:1011A000EAFFFF0EEE1801E1ED505EE10D50E66E34
:1011B00029EC12F0E5520001EC510D02F350E66EFD
:1011C000D950030FE96EDACFEAFFE552E750EE6E31
:1011D000ED6AD950030FE96EDACFEAFFEE50ED1059
:1011E00042E08A9A8A8C8A9C8A8C8A9C8A8C8A9C05
:1011F00000008A8A8A8C8A9C00008A9A8A8C8A9C3F
:101200008A8C8A9CEAC00DF00D5009E000000000B5
:10121000000000000000000000000D06F5D78A9ACB
:101220008A8C8A9C00008A8A8A8C8A9C8A8C8A9CF6
:101230008A8C8A9C00008A9A8A8C8A9C8A8C8A9CD6
:1012400006500D6E0D5009E0000000000000000087
:101250000000000000000D06F5D7030EDB06040EAB
:1012600001E2DB06B6D705D0FE0EE66E29EC12F0E1
:10127000E552F28E0DD0FE0EE66E29EC12F0E5522C
:101280000028EA6AA00FE96E000EEA22040EEF6E53
:1012900009EF12F0210EE66E29EC12F0E552020E73
:1012A0000024166E01010F51165C2CE2F29E8A8C0E
:1012B000939A8A9A8A9C8A8C8A9C8A8C8A9C8A8C29
:1012C0008A9C002A0050EA6AA00FE96E000EEA220A
:1012D000EFCF13F0002A0050EA6AA00FE96E000E6B
:1012E000EA22EFCF12F0110E0D6E0D4E08D0133220
:1012F0001232819AD8B0818A818C819CF6D78A9AE1
:10130000F28E0DD0FE0EE66E29EC12F0E5520028AA
:10131000EA6AA00FE96E000EEA22040EEF6E09EFF2
:1013200012F0220EE66E29EC12F0E552F29E8A8C43
:10133000939A8A9A8A9C8A8A8A8C8A9C8A9A8A8CAC
:101340008A9C8A8C8A9C8A8C8A9C8A8C8A9C8A8CAD
:101350008A9C8A8C8A9C8A8C8A9C8A8C8A9C8A8C9D
:101360008A9C8A8C8A9C938A090E0D6E0D4E07D03A
:10137000818C819CD89081BAD8801232F7D78A9A12
:10138000F28E12C0E6FF29EC12F0E55209EF12F0DE
:10139000230EE66E29EC12F0E552F29E8A8C939AA7
:1013A0008A9A8A9C8A8C8A9C8A8C8A9C8A8A8A8C51
:1013B0008A9C8A9A8A8C8A9C8A8C8A9C8A8C8A9C2F
:1013C0008A8C8A9C8A8C8A9C8A8C8A9C8A8C8A9C2D
:1013D0008A8C8A9C938A090E0D6E0D4E07D0818CE3
:1013E000819CD89081BAD8801232F7D78A9AF28E2F
:1013F00012C0E6FF29EC12F0E55209EF12F0240EBC
:10140000E66E29EC12F0E552002A0050EA6AA00FBD
:10141000E96E000EEA22EF500D6E01010F51005CE3
:1014200046E201500D24166E400E165C40E20D504F
:10143000E66E29EC12F0E552050E0DC0DBFF050E3D
:10144000DB5034E0F29E8A8C939A8A8A8A9C8A9A2C
:101450008A8C8A9C8A8C8A9C8A8A8A8C8A9C8A9AA0
:101460008A8C8A9C8A8C8A9C8A8C8A9C8A8C8A9C8C
:101470008A8C8A9C8A8C8A9C8A8C8A9C8A8C8A9C7C
:10148000938A090E0D6E0D4E07D0818C819CD890E9
:1014900081BAD8801232F7D78A9AF28E12C0E6FF4C
:1014A00029EC12F0E552050EDB06C9D70DD0FE0E71
:1014B000E66E29EC12F0E5520028EA6AA00FE96E08
:1014C000000EEA22040EEF6E09EF12F0250EE66E12
:1014D00029EC12F0E552020E0024166E01010F51A4
:1014E000165C2DE2F29E8A8C939A8A9A8A9C8A8C48
:1014F0008A9C8A8A8A8C8A9C8A8C8A9C002A0050C0
:10150000EA6AA00FE96E000EEA22EFCF13F0002A7C
:101510000050EA6AA00FE96E000EEA22EFCF12F047
:10152000110E0D6E0D4E08D013321232819AD8B0C2
:10153000818A818C819CF6D78A9AF28E0DD0FE0E1C
:10154000E66E29EC12F0E5520028EA6AA00FE96E77
:10155000000EEA22040EEF6E09EF12F0260EE66E80
:1015600029EC12F0E552002A0050EA6AA00FE96E59
:10157000000EEA22EF500D6E00500D240D24166E61
:1015800001010F51165C37E2060E0DC0DBFF060E9F
:10159000DB5030E0F29E8A8C939A8A8A8A9C8A9ADF
:1015A0008A8C8A9C8A8A8A8C8A9C8A8C8A9C002A49
:1015B0000050EA6AA00FE96E000EEA22EFCF13F0A6
:1015C000002A0050EA6AA00FE96E000EEA22EFCF6F
:1015D00012F0110E0D6E0D4E08D013321232819A98
:1015E000D8B0818A818C819CF6D78A9AF28E060EB9
:1015F000DB06CDD70DD0FE0EE66E29EC12F0E552DB
:101600000028EA6AA00FE96E000EEA22040EEF6ECF
:1016100009EF12F0270EE66E29EC12F0E552040EE7
:101620000024166E01010F51165C66E2F29E8A8C50
:10163000939A8A8A8A9C8A8C8A9C8A8C8A9C8A8CB5
:101640008A9C002A0050EA6AA00FE96E000EEA2286
:10165000EFCF13F0002A0050EA6AA00FE96E000EE7
:10166000EA22EFCF12F0110E0D6E0D4E08D013329C
:101670001232819AD8B0818A818C819CF6D78A9A5D
:101680008A8C8A9C8A8C8A9C8A8C8A9C8A8C002A66
:101690000050EA6AA00FE96E000EEA22EFCF13F0C5
:1016A000002A0050EA6AA00FE96E000EEA22EFCF8E
:1016B00012F01250131008E00000000000000000BB
:1016C0001206000E135AF5D78A9CEAC00DF00D5091
:1016D00009E0000000000000000000000000000021
:1016E0000D06F5D7100E0D6E0D5004E08A8C8A9C05
:1016F0000D06FAD7F28E0DD0FE0EE66E29EC12F032
:10170000E5520028EA6AA00FE96E000EEA22040EF4
:10171000EF6E09EF12F0280EE66E29EC12F0E5529A
:10172000040E0024166E01010F51165C67E2F29E52
:101730008A8C939A8A9A8A9C8A8A8A8C8A9C8A8CB6
:101740008A9C8A8C8A9C002A0050EA6AA00FE96E63
:10175000000EEA22EFCF13F0002A0050EA6AA00F31
:10176000E96E000EEA22EFCF12F0110E0D6E0D4E53
:1017700086D713321232819AD8B0818A818C819CAB
:10178000F6D78A9A8A8C8A9C8A8C8A9C8A8C8A9CB4
:101790008A8C002A0050EA6AA00FE96E000EEA2245
:1017A000EFCF13F0002A0050EA6AA00FE96E000E96
:1017B000EA22EFCF12F01250131008E000000000F0
:1017C000000000001206000E135AF5D78A9CEAC0EA
:1017D0000DF00D5009E000000000000000000000C6
:1017E000000000000D06F5D7F28E100E0D6E0D50A4
:1017F00003E08A8C0D06FBD78A9C0DD0FE0EE66EA8
:1018000029EC12F0E5520028EA6AA00FE96E000EFA
:10181000EA22040EEF6E09EF12F0290EE66E29ECB3
:1018200012F0E552030E0024166E01010F51165CF2
:1018300038E2002A0050EA6AA00FE96E000EEA22A0
:10184000EFCF12F0F29E8A8C939A050E0D6E0D4E1C
:1018500007D01232819AD8B0818A818C819CF7D7C7
:10186000002A0050EA6AA00FE96E000EEA22EFCFCC
:1018700013F0002A0050EA6AA00FE96E000EEA2277
:10188000EFCF12F0110E0D6E0D4E08D01332123242
:10189000819AD8B0818A818C819CF6D78A9AF28EFF
:1018A0000DD0FE0EE66E29EC12F0E5520028EA6A31
:1018B000A00FE96E000EEA22040EEF6E09EF12F09F
:1018C0002A0EE66E29EC12F0E5520028166E010190
:1018D0000F51165C3BE2002A0050EA6AA00FE96E45
:1018E000000EEA22EFCF12F0F29E8A8C939A050E38
:1018F0000D6E0D4E07D01232819AD8B0818A818C3C
:10190000819CF7D78A8C8A9C8A8C8A9C8A8C8A9C38
:101910008A8C8A9C8A8C8A9C8A8C8A9C8A8C8A9CD7
:101920008A8C8A9C938A090E0D6E0D4E07D0818C8D
:10193000819CD89081BAD8801232F7D78A9AF28ED9
:1019400012C0E6FF29EC12F0E5520DD0FE0EE66E55
:1019500029EC12F0E5520028EA6AA00FE96E000EA9
:10196000EA22040EEF6E09EF12F02B0EE66E29EC60
:1019700012F0E5520028166E01010F51165C43E289
:10198000002A0050EA6AA00FE96E000EEA22EF502A
:101990000D6EFF0E0D5C05E1C66A010E936E948C10
:1019A00031D0800EC76E080EC66EC56A0DBCC79ECC
:1019B000C70E936E8A6A0DB08A860DB28A880DB4FE
:1019C0008A8A949C8B9C380E0D160D5003E1770E7D
:1019D000C86E17D0080E0D5C03E13B0EC86E11D027
:1019E000100E0D5C03E1270EC86E0BD0180E0D5CB7
:1019F00003E10E0EC86E05D0200E0D5C02E10B0E49
:101A0000C86EC68A0DD0FE0EE66E29EC12F0E552C5
:101A10000028EA6AA00FE96E000EEA22040EEF6EBB
:101A200009EF12F02C0EE66E29EC12F0E552030ECF
:101A30000024166E01010F51165C01E3BDD0002A8F
:101A40000050EA6AA00FE96E000EEA22EF500D6E18
:101A50000001010E136E002A0050EA6AA00FE96E21
:101A6000000EEA22EFCF12F0C750040B01E0010E86
:101A7000166E1F0EC514161001E0F6D7C580C5B04E
:101A8000FED70D505DE0FE0E00011214C96EC7B006
:101A9000FED7C750040B01E0010E166E1F0EC514D1
:101AA000161001E0F6D7C5BC4AD0002A0050EA6AF9
:101AB000A00FE96E000EEA22EF50C96EC7B0FED744
:101AC000C750040B01E0010E166E1F0EC514161050
:101AD00001E0F6D7C5BC33D0C582C5B2FED7010E32
:101AE00000011210C96EC7B0FED7C750040B01E049
:101AF000010E166E1F0EC514161001E0F6D7C5BCF8
:101B00001ED00001136A0D50E66E29EC12F0E5526A
:101B10000D5011E0C586C7A0FED7C950E66E29EC6E
:101B200012F0E5520D50010804E2C59AC588C5B807
:101B3000FED70D06EDD7C58AC588C5B8FED725D016
:101B4000010E00011210C96EC7B0FED7C750040BBA
:101B500001E0010E166E1F0EC514161001E0F6D737
:101B6000C5BC13D00001136A010EE66E29EC12F019
:101B7000E552C586C7A0FED7C950E66E29EC12F023
:101B8000E552C58AC588C5B8FED7C550400B10E0E0
:101B9000000113500DE0FD0EE66E29EC12F0E55247
:101BA0000028EA6AA00FE96E000EEA22040EEF6E2A
:101BB000C584C5B4FED70DD0FE0EE66E29EC12F03A
:101BC000E5520028EA6AA00FE96E000EEA22040E30
:101BD000EF6E09EF12F02E0EE66E29EC12F0E552D0
:101BE000040E0024166E01010F51165C01E3A9D00A
:101BF000002A0050EA6AA00FE96E000EEA22EF50B8
:101C00000D6E0001010E136E002A0050EA6AA00F4B
:101C1000E96E000EEA22EFCF12F0C750040B01E08C
:101C2000010E166E1F0EC514161001E0F6D7C58002
:101C3000C5B0FED7FE0E00011214C96EC7B0FED7A4
:101C4000C750040B01E0010E166E1F0EC5141610CE
:101C500001E0F6D7C5BC5FD0002A0050EA6AA00FA9
:101C6000E96E000EEA22EF50C96EC7B0FED7C7502A
:101C7000040B01E0010E166E1F0EC514161001E0D4
:101C8000F6D7C5BC48D0002A0050EA6AA00FE96E1A
:101C9000000EEA22EF50C96EC7B0FED7C750040B42
:101CA00001E0010E166E1F0EC514161001E0F6D7E6
:101CB000C5BC31D0C582C5B2FED7010E00011210DD
:101CC000C96EC7B0FED7C750040B01E0010E166EF7
:101CD0001F0EC514161001E0F6D7C5BC1CD00001BC
:101CE000136A0D50E66EB5DBE5520D5010E0C58667
:101CF000C7A0FED7C950E66EACDBE5520D50010817
:101D000004E2C59AC588C5B8FED70D06EED7C58AC8
:101D1000C588C5B8FED7C550400B0FE00001135071
:101D20000CE0FD0EE66E95DBE5520028EA6AA00F96
:101D3000E96E000EEA22040EEF6EC584C5B4FED72C
:101D40000CD0FE0EE66E85DBE5520028EA6AA00F95
:101D5000E96E000EEA22040EEF6E5BD32D0EE66EE6
:101D600078DBE552002A0050EA6AA00FE96E000E07
:101D7000EA22EF500D6E020E00240D24166E0101B2
:101D80000F51165C71E2C750040B01E0010E166E94
:101D90001F0EC514161001E0F6D7C580C5B0FED7DA
:101DA000002A0050EA6AA00FE96E000EEA22EF5006
:101DB000FE0BC96EC7B0FED7C750040B01E0010E81
:101DC000166E1F0EC514161001E0F6D7C5BC37D02D
:101DD000002A0050EA6AA00FE96E000EEA22EF50D6
:101DE000C96EC7B0FED7C750040B01E0010E166ED6
:101DF0001F0EC514161001E0F6D7C5BC20D00D503B
:101E0000E66E27DBE5520D501AE0C550400B17E196
:101E1000002A0050EA6AA00FE96E000EEA22EF5095
:101E2000C96EC7B0FED7C750040B01E0010E166E95
:101E30001F0EC514161001E0F6D70D06E4D70D509D
:101E400003E1C550400B0CE0FD0EE66E02DBE552EF
:101E50000028EA6AA00FE96E000EEA22040EEF6E77
:101E6000C584C5B4FED70CD0FE0EE66EF2DAE5529C
:101E70000028EA6AA00FE96E000EEA22040EEF6E57
:101E8000C8D22F0EE66EE5DAE5520028166E010183
:101E90000F51165C37E2002A0050EA6AA00FE96E83
:101EA000000EEA22EF500D6EFF0E0D5C06E1C66AD1
:101EB000010E936E948C948E24D0C76A030EC66E66
:101EC0000DB6C6880DA4C78C0DB8C78EE50E936EEF
:101ED000949C949E030E0D160D5003E13B0ECB6EA9
:101EE0000DD00D0403E11D0ECB6E08D0020E0D5C6B
:101EF00003E10B0ECB6E02D0050ECB6E040ECA6E44
:101F0000C68A0CD0FE0EE66EA4DAE5520028EA6A14
:101F1000A00FE96E000EEA22040EEF6E7AD2300EA8
:101F2000E66E97DAE5520028166E01010F51165C35
:101F300020E2002A0050EA6AA00FE96E000EEA22B1
:101F4000EF500D6E0D50E66E84DAE5520D5005E14E
:101F5000C950E66E7EDAE5520BD00D5009E0C96A31
:101F6000C7A0FED7C950E66E74DAE5520D06F5D764
:101F70000CD0FE0EE66E6DDAE5520028EA6AA00F7C
:101F8000E96E000EEA22040EEF6E43D2310EE66EC9
:101F900060DAE552002A0050EA6AA00FE96E000EEE
:101FA000EA22EF500D6E00500D24166E01010F5104
:101FB000165C15E20D50E66E4CDAE5520D500EE05F
:101FC0009E96002A0050EA6AA00FE96E000EEA22EF
:101FD000EF50C96E9EA6FED70D06F0D70CD0FE0EB0
:101FE000E66E37DAE5520028EA6AA00FE96E000EC5
:101FF000EA22040EEF6E0DD2320EE66E2ADAE552B8
:10200000020E0024166E01010F51165C21E2002A17
:102010000050EA6AA00FE96E000EEA22EF508A6EC5
:10202000002A0050EA6AA00FE96E000EEA22EF5083
:102030000D6EC00E0D14166E3F0E8B1416108B6EA7
:10204000380E0D14166EC70E89141610896E0CD03A
:10205000FE0EE66EFED9E5520028EA6AA00FE96E90
:10206000000EEA22040EEF6ED4D1330EE66EF1D9E3
:10207000E552030E0024166E01010F51165C69E251
:10208000002A0050EA6AA00FE96E000EEA22EF5023
:102090000D6E002A0050EA6AA00FE96E000EEA22D7
:1020A000EFCF13F0002A0050EA6AA00FE96E000E8D
:1020B000EA22EFCF12F001500D240D24166E400ECF
:1020C000165C3AE20D50E66EC4D9E5520D5033E08D
:1020D0009E96200EC96E9EA6FED79E9613C0C9FF7F
:1020E0009EA6FED79E9612C0C9FF9EA6FED79E96BC
:1020F000C96A9EA6FED7C950E66EABD9E5529E9638
:10210000280EC96E9EA6FED79E9613C0C9FF9EA636
:10211000FED79E9612C0C9FF9EA6FED79E96C96A9C
:102120009EA6FED7C950E66E94D9E552122A000E3B
:1021300013220D06CBD70CD0FE0EE66E8AD9E552DF
:102140000028EA6AA00FE96E000EEA22040EEF6E84
:102150000CD0FE0EE66E7DD9E5520028EA6AA00F8B
:10216000E96E000EEA22040EEF6E53D1340EE66ED5
:1021700070D9E552002A0050EA6AA00FE96E000EFD
:10218000EA22EF500D6E00500D240D24020F166E42
:1021900001010F51165C54E20D50E66E5AD9E5521A
:1021A000002A0050EA6AA00FE96E000EEA22EFCF83
:1021B00013F0002A0050EA6AA00FE96E000EEA222E
:1021C000EFCF12F00D503BE09E96400EC96E9EA6DA
:1021D000FED79E9613C0C9FF9EA6FED79E9612C03C
:1021E000C9FF9EA6FED79E96002A0050EA6AA00F5D
:1021F000E96E000EEA22EF50C96E9EA6FED79E96AB
:10220000480EC96E9EA6FED79E9613C0C9FF9EA615
:10221000FED79E9612C0C9FF9EA6FED79E96002AA4
:102220000050EA6AA00FE96E000EEA22EF50C96E74
:102230009EA6FED7122A000E13220D06C3D70CD07D
:10224000FE0EE66E06D9E5520028EA6AA00FE96E96
:10225000000EEA22040EEF6EDCD0350EE66EF9D8E1
:10226000E5520028166E01010F51165C3BE2002A70
:102270000050EA6AA00FE96E000EEA22EF500D6EE0
:10228000FF0E0D5C05E1BA6ABD6A8A96B16A29D073
:1022900094849396B36AB26AC10EB16EBC6ABF6A87
:1022A0000D5003E13B0EBE6E16D00D0403E11D0E72
:1022B000BE6E11D0020E0D5C03E10B0EBE6E0BD094
:1022C000030E0D5C03E1050EBE6E05D0040E0D5C21
:1022D00002E1020EBE6E010EBB6E0B0EBD6E020E53
:1022E000BA6E0CD0FE0EE66EB4D8E5520028EA6A4B
:1022F000A00FE96E000EEA22040EEF6E8AD000688D
:1023000088D0F00EE66EA5D8E552020E0024166EB7
:1023100001010F51165C25E2002A0050EA6AA00F65
:10232000E96E000EEA22EFCF13F0002A0050EA6AAD
:10233000A00FE96E000EEA22EFCF12F013C0E6FF05
:1023400088D8E55212C0E6FF84D8E55213C0EAFFF0
:1023500012C0E9FFEF500D6E0D50E66E7AD8E552CF
:102360000CD0FE0EE66E75D8E5520028EA6AA00F82
:10237000E96E000EEA22040EEF6E4BD0F10EE66E0F
:1023800068D8E552030E0024166E01010F51165C49
:102390002EE2002A0050EA6AA00FE96E000EEA223F
:1023A000EFCF13F0002A0050EA6AA00FE96E000E8A
:1023B000EA22EFCF12F0002A0050EA6AA00FE96E7D
:1023C000000EEA22EF500D6E13C0E6FF42D8E55230
:1023D00012C0E6FF3ED8E5520D50E66E3AD8E552FF
:1023E00013C0EAFF12C0E9FF0D50EF6E0CD0FE0ED5
:1023F000E66E2FD8E5520028EA6AA00FE96E000EBB
:10240000EA22040EEF6E05D0FE0EE66E22D8E552EB
:1024100000D0002A01010F51005C11E3400EE66E6E
:10242000A00EE66E000EE66E6DEC16F0E552E5527B
:10243000E55201010F6F01010F5101E0006A070E23
:10244000E15C02E2E16AE552E16EE552E7CFD9FFD5
:102450001200D9CFE6FFE1CFD9FF010110510AE008
:102460000A0E025C11E20250022AEA6AE00FE96EEB
:10247000000E06D00150012AEA6A600FE96E000ED4
:10248000EA22FE0EDBCFEFFF400E015C13E1016A92
:1024900004010CBF0CD0400EE66E600EE66E000E1E
:1024A000E66E33EC16F0E552E552E55203D0010139
:1024B000010E106FE552E7CFD9FF1200D8CFE4FF2D
:1024C000E0CFE4FFE46EDACFE4FFE2CFDAFFF3CF50
:1024D000E4FFF4CFE4FFE652C2B2FED79E9C07C0F1
:1024E00009F008C00AF0C4CF08F0C3CF07F00B50C2
:1024F000075E0C50085AE10E0902F4CF0FF0F3CF3B
:102500000EF0E10E0A02F3500F260E5003260F5074
:102510000422E40E0702F4CF0FF0F3CF0EF0E40E26
:102520000802F3500F260E50035E0F50045A0001AC
:10253000043402E3036A046A05500001D88004549D
:1025400002E205C004F004C0BEFF00010350E840F1
:10255000E8403F0B300B186ECF0EBD141810BD6E47
:10256000E552E5CFF4FFE5CFF3FFE5CFDAFFE55025
:0A257000E5CFE0FFE5CFD8FF100033
:06257A006C5002E0000EAF
:1025800001D0010E00090BE0040100513C0BE842B0
:10259000E8420D0802E1D8EF12F00DEF13F06C5095
:1025A00002E0000E01D0010E040901E045D812003E
:1025B000D9CFE6FFE1CFD9FFE6520101006B016BF5
:1025C000066B076B34EC14F0DF6ADF50166E176A87
:1025D000010E165C000E17581AE20101015117E1B5
:1025E000F76ADF34FE0BF736F66E930EF626300EE2
:1025F000F7220900F5CF16F00800F5CF17F004D048
:1026000017C0FAFF1650F96EFBDFDF2ADED7D9D8E4
:10261000E552E552E7CFD9FF1200020E0101005D3D
:1026200009E192D8040100BD02D0C80E01D0880E85
:10263000006F120026EF14F0040E0001FB5D09E1AB
:1026400012C46EFF6E50000802E2050E01D0030EA8
:10265000FB6F0101000509E10AD8040104BD02D0A5
:10266000C80E01D0880E046F120026EF14F0D9CFE7
:10267000E6FFE1CFD9FF020EE1260101080E065D5B
:10268000000E075905E206C1DEFF07C1DDFF03D0DA
:10269000080EDE6EDD6A040104930491010EDB5026
:1026A0000413DFCF05F4000EDB500101065F010EBD
:1026B000DB50075B180E046F040E056F0001FCA3CE
:1026C0001DD0D9CFE9FFDACFEAFFEE50ED1032E0AE
:1026D00002C1F6FF03C1F7FF0800F55004C1E9FF8E
:1026E00005C1EAFFEF6E0101042B000E0523022B4A
:1026F0000323DF06010EE5E2DB06E3D7D9CFE9FFCE
:10270000DACFEAFFEE50ED1015E002C1E9FF03C198
:10271000EAFFEF5004C1E9FF05C1EAFFEF6E0101D6
:10272000042B000E0523022B0323DF06010EE6E235
:10273000DB06E4D7020EE15C02E2E16AE552E16EFB
:10274000E552E7CFD9FF1200D9CFE6FFE1CFD9FF9D
:10275000020EE126030E04010015E76E010EE7CF1D
:10276000DBFF01C4DFFFDE5001010627DD50072338
:10277000180E026F040E036FD9CFE9FFDACFEAFF1C
:10278000EE50ED1014E002C1E9FF03C1EAFFEF5083
:1027900004C1E9FF05C1EAFFEF6E042B000E05231B
:1027A000022B0323DF06010EE7E2DB06E5D7020E6C
:1027B000E15C02E2E16AE552E16EE552E7CFD9FF62
:1027C0001200010101510BE10401080E016F100E0E
:1027D000026F040E036F840E006F040123D0040106
:1027E00010AF22D0010106510401165D010107510D
:1027F0000401175904E216C406F117C407F137DFC4
:102800000101010E006F0401080E016F100E026F2E
:10281000040E036F800E006F0401180E066F040E85
:10282000076FC80E046F10D00101020E006F040183
:10283000056BC80E046F0401080E016F180E026FBD
:10284000040E036FC80E006F6D9812000101006B3B
:102850000401080E016F100E026F040E036F880E44
:08286000006F0401046B12007B
:0828680004011051600BE8426D
:10287000E842E842E842E842000901E01200115152
:10288000070A4CE00B0A4AE0070A3BE0010A27E08E
:102890000B0A23E0020A21E0030A1DE0080A12E005
:1028A000010A0EE00F0A0AE0030A01E0120001012A
:1028B000010E016F0001040EFB6F12008FEF14F088
:1028C000E6EF14F00101010E016F0101FD0E026F30
:1028D000000E036F10D00DEF15F058EF15F0010149
:1028E000010E016F040114510101026F036BFE0E12
:1028F0000227000E03230001FC930101010E066F65
:1029000012000101010E016F04011451EA6AFE0F69
:10291000E96E000EEA2212C4EFFF12001200800ED0
:102920000401105D52E11351030A30E0010A0CE08A
:10293000030A49E10101010E016F0101D60E026F88
:102940002F0E036F120E3CD00101010E016F040126
:102950001251F66EF76AD890F636F736890EF626DB
:10296000300EF7220900F5CF02F10A00F5CF03F18E
:10297000020E0101F76A0225F66E0351F7220900E3
:10298000F5CF06F10A00F5CF07F11DD00101010EC8
:10299000016F04011251F66EF76AD890F636F736D9
:1029A0008D0EF626300EF7220900F5CF02F10A004F
:1029B000F5CF03F102C1F6FF03C1F7FF0800F550A0
:1029C0000101066F076B0001FC8312000101010E7B
:1029D000016F0F0EE66E710EE66E0F0EE66E57EC8F
:1029E00017F0E552E552E552010EE66EFE0EE66E78
:1029F000000EE66E57EC17F0E552E552E55212C4B0
:102A0000FDF00401125104E10001050EFB6F1200FC
:102A10000001060EFB6F1EEF16F00401186B196B18
:102A2000040110511F0B020A13E0030A0DE0010A12
:102A300031E10101010E016F040118810001FCA1C7
:102A400029D00401188326D00101010E016F22D084
:102A50000101010E016F040114510F0B080DF35019
:102A6000176A000F166E040E17221451800B01E036
:102A7000010E040DF35001011624046F000E1720FF
:102A8000056F04C1E9FFEA6EEF50040B03E0040197
:102A9000010E186F010101050AE10101180E026F14
:102AA000040E036F0001FC930101020E066F120079
:102AB0000401120510E110511F0B00090CE1010186
:102AC000010E016F030E0401115D03E10001FC81A1
:102AD00002D00001FC91040112513AE110511F0B88
:102AE000020836E114510F0B000932E00101010E1A
:102AF000016F040114510F0B080DF350176A000FFA
:102B0000166E040E17221451800B01E0010E040D05
:102B1000F35001011624046F000E1720056F030EF9
:102B20000401115D07E1840E04C1E9FF05C1EAFF5C
:102B3000EF6E120014AF06D004C1E9FF05C1EAFF31
:102B4000EF6A1200880E04C1E9FF05C1EAFFEF6ECB
:022B5000120071
:0E2B5200040110511F0B010801E01200145184
:102B600001E01200060E115D28E11351230A23E053
:102B7000010A0FE0030A1FE10101020E016F0001CB
:102B8000FD0505E10101FA0E026F2F0E036F090E1C
:102B90000FD00101020E016F0001FD0505E10101E9
:102BA000670E026F300E036F0001FD0504E1220E77
:102BB0000101066F076B0001FC8304011051600BDB
:102BC000E842E842E842E842E842010801E0120037
:102BD00011510B0A2BE0080A1BE0090A13E0080A4E
:102BE00009E00B0A05E0080A01E012001CEF16F0EC
:102BF0001DEF16F00101020E016F0101080E026FB8
:102C0000010E0DD00101020E016F13C408F1120074
:102C10000101020E016F0101090E026F010E036F27
:102C20000001FC930101010E066F12000101020E6A
:102C3000016F12C409F112001200120001010A6BA7
:102C40001E0E716E0401400E096F200E0A6F040EF5
:102C50000B6F880E086F0401600E0E6F040E0F6F6D
:102C6000400E0C6F1200D9CFE6FFE1CFD9FFE6523C
:102C7000FC0EDB50400805E2400EF36EFC0EF3CF75
:102C8000DBFFDF6AFC0EDB50DF5C19E2DF50E76E32
:102C9000FD0EDBCFE9FFFE0EDBCFEAFFE750E926B2
:102CA000000EEA22EF50E66EDF50EA6A600FE96E2E
:102CB000040EEA22E552E750EF6EDF2AE3D7FC0E5E
:102CC000DBCF0DF4400E04010C170C7D880E0C13A5
:102CD000E552E552E7CFD9FF1200D9CFE6FFE1CFA9
:102CE000D9FF01010A6B040108BF30D0FC0EDBCF15
:102CF00016F00951D880165403E2FC0E09C4DBFF1C
:102D000001010A6BFC0EDB500A5D19E20A51EA6A06
:102D1000200FE96E040EEA22EF50E66E0A51E76ECC
:102D2000FD0EDBCFE9FFFE0EDBCFEAFFE750E92621
:102D3000000EEA22E552E750EF6E0A2BE3D70401BA
:102D4000400E096F0817087D880E081301010A510B
:082D5000E552E7CFD9FF1200A4
:082D58006DA60CD80001FB057B
:102D600008E16DBA06D0686A696A69806988020EEE
:102D7000FB6F12006D6A696A6D860001010EFB6FC0
:102D800012006D6A696A0001FB6B1200C1EF16F058
:102D90000001FB5101E112006850040B04E069508E
:102DA000040B01E041D86DB212006850010B04E041
:102DB0006950010B01E059D86850100B04E06950CC
:102DC000100B01E024D86850400B04E06950400B20
:102DD00001E040D86850200B04E06950200B01E06E
:102DE0003BD86850020B04E06950020B01E03BD86D
:102DF000030E0001FB5D01E212006850080B06E0C3
:102E00006950080B03E0BDEC12F06896120069846B
:102E100068986D82A19AF290A08AF2860300F2B0BF
:102E200007D8A09AF29612006D92699468941200E5
:102E30000001FCA10ED0F8DF6D840101080E0B6FBC
:102E4000070E0C6F0B07000E0C5B0B510C11FAE117
:102E50006D941200689C120070A003D026EC14F050
:102E60007090689A1200689212006A6A686A9F0EEF
:102E70006B6E7B0E696E6E6A0F0EE66E710EE66EFD
:102E80000F0EE66E14D8E552E552E552160E706E3E
:102E900068A602D06896FCD76D9826EC14F0000165
:102EA000FC910001FD6B0001030EFB6F1200D9CFF6
:102EB000E6FFE1CFD9FFFD0EDBCFE9FFFE0EDBCF52
:102EC000EAFFFC0EDB5004E0EE6AFC0EDB06F9D7ED
:082ED000E552E7CFD9FF120023
:082ED800D9CFE6FFE1CFD9FFDD
:102EE000E65204011351030A1DE0010A1DE18A7430
:102EF000125118E1010EDF6EDF50400813E3DF04CA
:102F0000EA6A200FE96E040EEA22EF50E66EDF0453
:102F1000EA6A600FE96E040EEA22E552E750EF6EAE
:102F2000DF28E9D704011251E552E552E7CFD9FF76
:102F3000120001010D510E1104E1100E0D6F270E4C
:102F40000E6F0D07000E0E5B6DA208D00D510E1115
:102F500030E189728950020B13E128D00001FB5146
:102F600002E1899223D0FB0502E1898209D0020E99
:102F7000FB5D02E189821AD0030EFB5D03E18992B9
:102F800089841200050EFB5D06E101010D510E1151
:102F900010E189720BD0060EFB5D0BE101010D51B2
:102FA0000E1107E189728950020B02E08994120028
:102FB00089841200D9CFE6FFE6520101600E026F4C
:102FC000040E036F0101400E066FE552E552E7CF94
:062FD000D9FF12001200FF
:0A2FD6001201000200000008D804F8
:102FE000000101000102000109022900010100A005
:102FF000140904000002030000000921010100017E
:10300000222200070581034000010705010340005B
:10301000010403090414034F00700065006E0020D2
:1030200000500072006F0067003E034F00700065A3
:10303000006E002000500072006F00670072006197
:10304000006D006D006500720020002000550053E7
:103050000042002000480049004400200063006C4A
:103060000061007300730006A0FF0901A1010903BC
:10307000150026FF007508954081020904150026F9
:10308000FF00750895409102C0E82FE82F11301518
:05309000302930522B35
:0A3096002A0EF66E000EF76E000E13
:1030A000F86E00010900F550F66F0900F550F76F52
:1030B00003E1F66701D03DD00900F550F16F09003A
:1030C000F550F26F0900F550F36F09000900F55053
:1030D000E96E0900F550EA6E090009000900F55093
:1030E000F46F0900F550F56F09000900F6CFF8F00C
:1030F000F7CFF9F0F8CFFAF0F1C0F6FFF2C0F7FF22
:10310000F3C0F8FF0001F45302E1F55307E00900B2
:10311000F550EE6EF407F8E2F507F9D7F8C0F6FFC0
:10312000F9C0F7FFFAC0F8FF0001F607000EF75BE1
:04313000BFD71200F3
:0C31340009D8ACEC16F06FBE02D0C8EC5D
:1031400016F047EC00F0F7D70F0EC112140E6F6E99
:103150000001FB6B0001FC6B0001FD6B28EF00F030
:1031600013EE00F023EE00F0F86A159C4BEC18F01B
:0C317000C5EC18F09AEC18F0FBD7120028
:04317C0000EE00F071
:0A3180000F0EEE6AEA62FDD712009E
:02318A00120031
:04318C00000000003F
:1031900000640100000000AB03000000000000001C
:0231A00000002D
:0231A20000002B
:020000040030CA
:0100000022DD
:010001000EF0
:010002003DC0
:010003001EDE
:0100050000FA
:010006008178
:0200000400F00A
:100000004F70656E2050726F6772616D6D65722002
:10001000762E20302E352E30202D20436F707972B1
:100020006967687420284329203230303820416CB9
:10003000626572746F204D616363696F6E69202D14
:100040002054686973206973206672656520736F38
:070050006674776172650020
:00000001FF
